:100000000C942A000C9447000C9447000C94470071
:100010000C9447000C9447000C9447000C94470044
:100020000C9447000C9447000C9447000C94470034
:100030000C9447000C9447000C9447000C94470024
:100040000C9447000C9447000C9447000C94470014
:100050000C94470011241FBECFE5D4E0DEBFCDBF16
:1000600010E0A0E6B0E0E0E2F1E002C005900D9201
:10007000A036B107D9F710E0A0E6B0E001C01D92AC
:10008000A036B107E1F70E9457000C948F000C9442
:100090000000CF93DF93CDB7DEB7E8E3F0E0108246
:1000A000E7E3F0E081E08083DF91CF910895CF9383
:1000B000DF93CDB7DEB724970FB6F894DEBF0FBE3F
:1000C000CDBF0E944900A8E3B0E0E8E3F0E0808102
:1000D00081608C9380E593EC9C838B8305C08B813E
:1000E0009C8101979C838B838B819C810097B9F7BE
:1000F000A8E3B0E0E8E3F0E090818EEF89238C93F1
:1001000080E593EC9C838B8305C08B819C81019758
:100110009C838B838B819C810097B9F7D4CFFFCFD1
:00000001FF
